:1000000021288E0032308D0032308C008C0B062877
:100010008D0B04288E0B0228080085308400FF30E9
:10002000800086308400FF30800008008530840026
:10003000FB308000FB30850086308400003080007B
:1000400008000D2006088F0003118F09031960288E
:10005000890106088F0003118F0903192928060852
:100060008F0016200F0886002F3001200D20060873
:1000700003118F02031D29288800831608155530A7
:100080008900AA308900881488184428081183122E
:1000900089195728890A162086010F3001200D2062
:1000A00006088F0003118F09031929284B281620F1
:1000B000860105300120FF308600053001205828D8
:1000C00016208901831608148312080886001F3041
:0A00D000012089196128890A6228BD
:02400E00F13F80
:00000001FF
